:1001000012010002000000400516108001000102EB
:020110000001EC
:0A0114000A0600020000004001008E
:1001200009022000010100A0FA0904000002FF00FA
:100130000000070502020002000705860200020017
:1001420009022000010100A0FA0904000002FF00D8
:10015200000007050102400000070581024000007F
:100164001403000000000000000000000000000074
:1001740000000000260341004300430045005300F3
:10018400200049002F004F002000500072006F0033
:100194006400750063007400730026035500530067
:1001A40042002D004900440049004F002D00310059
:1001B40036002000460061006D0069006C00790083
:1001C40000008081828384858687909192939495A0
:1001D4009697A0A1A2A3A4A5A6A7B0B1B2B3B4B5A3
:1001E400B6B7C0D0C0E0EF9001C6939001FDF0ED2A
:1001F4009001C6939001FFF0A2009200D0E0D0D00D
:1002040022C0D0C0E0EF9001C69390021CF0ED90A4
:1002140001C69390021FF0A200B39200D0E0D0D0A8
:0102240022B7
:100056005553422D4949524F2D3136005553422DA5
:1000660049492D3136005553422D524F2D31360018
:100076005553422D4949524F2D38005553422D496B
:10008600492D38005553422D4949524F2D303400E1
:100096005553422D4944494F2D3136005553422D73
:1000A60049492D31362D4F454D005553422D494472
:1000B6004F2D3136005553422D4944494F2D3800B6
:1000C6005553422D49492D382D4F454D0055534224
:1000D6002D4944494F2D34005553422D49492D345D
:1000E6002D4F454D005553422D49492D4F544845F6
:0200F6005200B6
:1018FA0090E740E580F0A3E590F0A3E5A0F0A3E52A
:10190A00B0F0E42290E68AF090E6BEE090E68BF032
:08191A0090E6A0E04480F022F9
:0400460043B1402260
:04004E0053B1BF22C9
:041C5F0063B140220B
:071C580053B1F543B10A226C
:10158600EF5407FE7401A806088002C333D8FCFE98
:10159600EF131313541FFFED6011EF14600804706E
:1015A6001BEE42808016EE42908011EF1460090413
:0F15B600700AEEF452808004EEF45290021C583A
:100DC300EF54F824F8601024F8601024F86010241D
:100DD30018700EAE80800AAE908006AEA08002AE80
:100DE300B0EF5407FF7401A807088002C333D8FC8F
:0B0DF3005206EE60047F0180027F00CA
:010DFE0022D2
:10000E00E58012083A900001E59012084C9000022B
:0D001E00E5A012084C900003E5B002084C6C
:101AF3001207F490205EF0F58090000112080D901B
:081B0300205FF0F590021C5870
:01004A002293
:031C6F00020C1B49
:01005200228B
:010DFF0022D1
:011C8500223C
:100C1B007AE779407F40AB077D017F037E00121698
:100C2B007690E740E0541FF55890010AE04558F0E4
:100C3B00E558540FB410004003020CE6900C4EF82C
:100C4B00282873020C7E020C86020C8E020CE60224
:100C5B000C96020C9E020CA6020CE6020CAE020CC9
:100C6B00B6020CBE020CE6020CC6020CCE020CD66F
:100C7B00020CDE7BFF7A00795680667BFF7A007967
:100C8B0062805E7BFF7A00796C80567BFF7A0079FD
:100C9B0076804E7BFF7A00798180467BFF7A0079E4
:100CAB008A803E7BFF7A00799680367BFF7A0079CB
:100CBB00A2802E7BFF7A0079B080267BFF7A0079A9
:100CCB00BB801E7BFF7A0079C680167BFF7A00798A
:100CDB00D3800E7BFF7A0079DE80067BFF7A00796A
:050CEB00EB1213712261
:091C230090205D74FFF0A3F02293
:101A120090205DE0F580A3E0F59075B2FF75B3FF0D
:0E1A2200E4F5B4F5B575B18A75B67F021C58AF
:101BAF008F248D253006030201E6AD25AF241202E6
:021BBF000522FD
:011C8600223B
:031C7200021C58F9
:091C2C0090206174FFF0A3F02286
:0D003600902061E0F580A3E0F590021C58D9
:1015C50090E6B8E030E7071218FA12190E2290E6F5
:1015D500BEE0D394004024E090E68BF090E6A0E0D6
:1015E50020E1F990E740E090205DF0F58090E7413B
:0C15F500E0FF90205EF0F590121C5822E0
:1018A600D204120B39402290E6B9E024D0600C1421
:1018B6006009241F70111215C5800E1218FA90E6E1
:0B18C600BAF012190E8002D322C322D8
:101AD8005641756720323520323031354031323A3F
:0B1AE80030343A3337000000000000EB
:101BC10002541AEF023F00000147010143010141A4
:011BD1000112
:1006A000E0FFAE30053074402EF582E434E7F58388
:1006B00022E490E68AF090E6BEE090E68BF022908D
:1006C000E740F0E490E68AF090E68B22FF7E000D92
:1006D000EE2555F582E43554F58322E0FE74892F2A
:1006E000F582E43420F583222530F530E533352FCB
:1006F000F52FC3E5329534F532E5319533F53122E6
:1007000074402536F58274E73535F5832224617C03
:10071000007B01F9EC22E52125E0240AF582E4348E
:1007200020F583E0FE547FFFEE225391EF90E65DCB
:100730002274692FF582E43420F5832274652EF546
:1007400082E43420F583E0227D657A207B007F01FE
:100750007E1F22E4F50BF50CF556F55722F0748D4B
:100760002FF582E43420F5832290E6BEE064012276
:10077000C3E5369534E53595332274912FF582E43F
:100780003420F58322F583EFF0052BE52B2290E64C
:10079000BEE0640222F583EFF090E741E0FFEE2532
:1007A000E022E5302536F582E52F3535F5832285C3
:1007B000090F850A108513118514122285130F85E0
:1007C0001410850911850A122290E6A0E04480F0F9
:1007D00022AD347AE77B40AF30AE2F227C007B0124
:1007E000F9EC2290201AE0FFE521C39F227B017AD9
:0407F000E779402243
:101B6300902003E07006902002E06003021C011243
:031B7300002E221F
:1019D1007E007F657D007B017A2079001208E99005
:1019E10020007409F0E4A3F0121C23121A12021B46
:0119F100E312
:1019F2007D0212074A121676902000E0B40904A371
:101A0200E060030219D1120748121676121A122246
:0F1BE3001207481217537D657F007E1F021C7585
:1012B700121B6390E6BEE0F530753202E530604BF5
:1012C700C39440500585303180037531401206C301
:1012D700E531F090E6A0E020E1F9E4F52FE52FC332
:1012E7009531501E7440252F1206A9E0FFAE320536
:1012F70032EE240012070F3420FAEF12083A052FB6
:0E13070080DBC3E5309531F53080B1021B6309
:1011030090E6B8E030E733E4F530F52FE52FC394EC
:101113000450207E007B01745D252FF9EE3420FA04
:101123001207F4FF744025301206A9EFF0052F05CE
:101133003080D91206B11207C9221206B690E6A072
:10114300E020E1F990E6BEE064046003C20422E417
:10115300F530F52FE52FC39404501D74402530124C
:1011630006A9E0FFE52F245D1207DC3420FAEF1215
:10117300083A052F053080DC90E6BAE0B4CE08A328
:07118300E0B4AC03121BE312
:01118A002242
:0F1BF200D3E5579545E55695444003121C35221F
:011C8700223A
:10194700902005E0FE902004E07C002400F545ECA3
:101957003EF54445457007C28CC2A9C20522D28C08
:03196700D2A922E0
:011C88002239
:10163C001206B690E6A0E020E1F9E4FF74422FF523
:10164C0082E434E7F583E0FEEF12070D3420FAEE66
:10165C0012083A0FBF04E590E740E0902004F090A8
:0A166C00E741E0902005F002194765
:091C3500120036120753D20522F9
:101B0B00C205120753C28CC2A9538EF75389F143F6
:081B1B008901121C8802194720
:1016E700E540453F6019E54015407002153F14C3BA
:1016F70094FFE53F64809480501612004E801130AD
:10170700040E753F057540FF120046C204120753C9
:05171700300502D204C0
:01171C0022AA
:100CF00090E6B8E030E75CE4F5309020041206A0FE
:100D0000EFF09020051206A0EFF0E4F52FE52FC3D9
:100D1000940450207E007B017461252FF9EE34206D
:100D2000FA1207F4FF744025301206A9EFF0052FE0
:100D3000053080D91206A2E557F0E5561206A1EF5C
:100D4000F0A205E4331206A1EFF0C2051206B112BB
:100D500007C9221206B690E6A0E020E1F9C205908C
:100D6000E6BEE064066003C20422E4F530AF30055D
:100D70003074402F1206A9E0902004F0AF30053007
:100D800074402F1206A9E0902005F0E4F52FE52F1E
:100D9000C39404501B744025301206A9E0FFE52FD0
:100DA00012070D3420FAEF12083A052F053080DEC5
:100DB00012194790E6BAE0B4CE08A3E0B4AC03122F
:020DC0001BE333
:010DC200220E
:041C6300754701229E
:10131500121B6390E6BEE0F530E4F532E530604B34
:10132500C39440500585303180037531401206C3A2
:10133500E531F090E6A0E020E1F9E4F52FE52FC3D3
:101345009531501E7440252F1206A9E0FFAE3205D7
:1013550032EE241B1207DC3420FAEF12083A052F6F
:0B13650080DBC3E5309531F53080B12E
:01137000225A
:1013C8001547E547704B90201BE0F547121C86E453
:1013D800F52190205CE0FFE521C39F5031E52125F0
:1013E800E0241CF582E43420F583E0F522E521258C
:1013F800E0241DF582E43420F583E0F523547FFDD5
:10140800E523339206AF22121BAF052180C4121CBC
:011418007261
:0114190022B0
:101AA2001206B690E6A0E020E1F990E740E090202F
:0B1AB20006F090E741E0902007F022D2
:101254001543E543705C902006E0F5437B017A205A
:10126400799512000EE4FFFE74952EF582E4342085
:10127400F583E0FD12073C6DF97D01E4FCECC394B9
:10128400085029E95D6013120731E014F0120731A8
:10129400E0701112073C6DF08000902007E0FB1213
:1012A4000731EBF00CED25E0FD0F80D10EEE640468
:0212B40070B612
:0112B6002215
:101B76001206B690E6A0E020E1F990E740E090205A
:031B860008F02242
:101B2300E4FF1206DDE4F012077A74FF12075DE4A6
:051B3300F00FBF04EDFE
:011B3800228A
:101545001541E541703A902008E0F5417B017A208C
:10155500798912000EE4FF12077AC083C082120651
:10156500DBE0FDEE5DD082D08312075DC083C082D3
:101575001206DBE0FDEE4DD082D083F00FBF04D71D
:011585002243
:041C6700754601229B
:10118B001546E5466027E4F5211207E35056744CEB
:10119B002521F8E6601316E6700F12071630E704E8
:1011AB007D0080027D01121586052180DC902009CF
:1011BB00E0F546E4F5211207E35029E52125E0246B
:1011CB000BF582E43420F583E0FF744C2521F8A65F
:1011DB000712071630E7047D0180027D0012158689
:0411EB00052180D288
:0111EF0022DD
:1018D1001206B690E6A0E020E1F9E4FF74402F1271
:1018E10006A9E0FEEF7C007B012409F9EC3420FA23
:0818F100EE12083A0FBF12E4E9
:0118F90022CC
:040FE9008E2F8F3088
:100FED00E4F531E5306402452F700C90E741F0E5F2
:100FFD003015307002152FE5306401452F701090BB
:10100D00E74074651206B5E53015307002152FE511
:10101D0030452F605490E6A0E020E1F9C3E530940F
:10102D0040E52F94005004AD3080027D40E4FFEF89
:10103D00C39D5021AE310531EE7583007B01240037
:10104D00F9E5833420FA1207F4FE74402F1206A935
:10105D00EEF00F80DA1206C3EDF0FFC3E5309FF519
:09106D0030E52F9400F52F80A658
:011076002257
:1002250090E6B8E030E76090E6BFE0FE90E6BEE01D
:10023500FDEDFF4E7002804A90E6BDE0FD90E6BC04
:10024500E04D7003020FE990E6BDE060030204F59E
:1002550090E6BCE01460030204F57532FF75331AAD
:100265007534D875350075361E7B017AE7794112EC
:10027500141A1207ED121B4EEF0490E740F090E6BA
:10028500BEE090E68BF02290E6BFE0FF90E6BEE090
:100295004F707790E6BDE0704D90E6BCE024EF60CE
:1002A50023249F603024FD603324F360342472706E
:1002B5003590E6BAE064CE702DA3E064AC702712E9
:1002C5001BE3802290E6BAE0B4CE1BA3E0B4AC16E3
:1002D5001219D18011E490201AF0800A7546018028
:1002E50005E490205CF090E6BDE0648060030204C4
:1002F500F590E6BCE0640160030204F590E6BAE01F
:10030500902002F090E6BB0203BC90E6BFE06003DC
:100315000204F590E6BDE0FE90E6BCE07C0024001A
:10032500FFEC3E60030204F5EF1208C303652003EA
:100335006521036522036523039A2F03C44103D274
:100345005103DD5303FA610405630422710430731C
:10035500044D74049181049C8304B684000004F563
:1003650090E6BEE0B463031212B790E6BCE030E05D
:1003750003121A1290E6BCE020E1030204F590E6B0
:10038500BAE064CE60030204F5A3E064AC60030246
:1003950004F5021BE312078E60030204F5E090E604
:1003A5008BF090E6A0E020E1F9121B6390E740E0B6
:1003B500902002F090E741E0902003F0021B63904B
:1003C500E6BEE0640660030204F502163C12078EE1
:1003D50060030204F5021AA212076960030204F51C
:1003E500E090E68BF090E6A0E020E1F990E740E0B0
:1003F500902006F02212076960030204F5021B76BD
:1004050012076960030204F5E090E68BF090E6A020
:10041500E020E1F990E740E0902008F02290E6BE68
:10042500E0641260030204F50218D1120769600343
:100435000204F5E090E68BF090E6A0E020E1F9906B
:10044500E740E0902009F02212078E60030204F5D0
:1004550090201AE0C3940840030204F51206B690F2
:10046500E6A0E020E1F990E740E0FF90201AE0FEE9
:1004750025E02408F582E434201207952409F58245
:10048500E43420F583EFF090201A806190E6BEE019
:100495006442705C0213151207697054E090E68B94
:1004A500F090E6A0E020E1F990E740E090201BF015
:1004B5002212078E703A90205CE0C39420503112CE
:1004C50006B690E6A0E020E1F990E740E0FF902035
:1004D5005CE0FE25E0241AF582E434201207952419
:1004E5001BF582E43420F583EFF090205CE004F006
:0104F50022E4
:101ABD0090E6047480F00000007402F000000074E1
:0B1ACD0006F0000000E4F00000002222
:011C89002238
:10160100E4F52A7AE779407F40AB077D087FF87ED1
:101611001D121676E4F52A7440252A1206A9E0FD6A
:10162100E52A75F002A42466F9740135F08982F582
:0A16310083EDF0052AE52AB408DD78
:01163B00228C
:1014B90090E678E05410FFC4540F4450F54813E403
:1014C90033F54A90E600E054E7F0438E2012002EEF
:1014D90012004A121C50121601121C6FD200121966
:1014E900F2121B0B121C63121B23121C67121B63C3
:0614F90012004E02005239
:101A3000120DFF1216E7121BF2E5B190E68020E7C7
:0E1A400006E04408F08004E054F7F0021C8534
:061371008B2A8A2B892C57
:10137700E4F52D121B4E8F2EE52E25E02402900159
:101387009EF0E4F52DAF2EEF3395E0FEC3E52D9FDC
:10139700EE6480F87480985027AB2AAA2BA92C8575
:1013A7002D8275830012080DFDE52D75F002A4242A
:1013B700A0F9740135F08982F583EDF0052D80C51C
:0113C7002203
:0616AF008E3D8F3EAC05EC
:1016B500E4FDE54A6007E53D1206CCEFF0AE050D09
:1016C500E5552E1206D3E53EF0AF050DE5552F1273
:1016D50006D3ECF0AB55AA54AF48121A86AF4802B0
:0216E500171DCF
:031C75000216AFA5
:0A1753008E378F388D398A3A8B3BB0
:10175D00E4F53CE53CC3953950200538E538AE3706
:10176D007002053714FFE53B253CF582E4353AF56B
:0A177D0083E0FD121C75053C80D9C5
:01178700223F
:0A1676008E378F388D398A3A8B3B8E
:10168000E4FDF53CE54A6007E5371206CCEFF0AE25
:10169000050DE5552E1206D3E538F0AB55AA54AF2B
:0F16A00048121A86AB3BAA3AAD39AF48021A6A14
:1009150090E6BAE0752F00F530A3E0FEEE422F9089
:10092500E6BEE0753100F532A3E0FEEE423190E619
:10093500B8E064C060030209DBE5324531700302AB
:100945000A3090E6A0E020E1F9C3E5329440E531B4
:10095500940050088531338532348006753300752F
:10096500344090E6B9E064A3704090E6BCE0B40181
:100975001BA3E0701790E6BBE030E71090E74074EA
:1009850003F0A37401F0A37403F0803EE4F535F59C
:100995003612077050341207A2E0FF120700EFF07D
:1009A5000536E53670EB053580E7E4F535F53612A5
:1009B5000770501012070074CDF00536E53670EF5C
:1009C500053580EB1207D11216761206C3E534F011
:1009D5001206E802093E90E6B8E06440704DE53243
:1009E500453160471206C3F090E6A0E020E1F9909A
:1009F500E68BE0753300F53490E6B9E0B4A31EE468
:100A0500F535F536120770501A120700E0FF120788
:100A1500A2EFF00536E53670EB053580E71207D114
:0B0A2500121753E5341206E80209E343
:010A300022A3
:0B1C0E00E54545447003D38001C3226C
:021C7B00D32272
:021C7D00D32270
:0800030090E6BAE0F542D322B9
:091C3E00E5421206BF04F0D322B6
:0800F80090E6BAE0F549D322BD
:091C4700E5491206BF04F0D322A6
:021C7F00D3226E
:021C8100D3226C
:021C8300D3226A
:100EB800E4FF90E6B8E020E703020F570F0F7440F5
:100EC80024011206A97409F00F744024021206A91D
:100ED800E4F00F744024031206A9E4F00F744024D0
:100EE800041206A9E4F00F744024051206A974043C
:100EF800F00F744024061206A9E4F00F744024078A
:100F08001206A9E4F00F744024081206A974FFF031
:100F18000F744024091206A974FFF00F7440240AC4
:100F28001206A97408F00F7440240B1206A9742045
:100F3800F00F7440240C1206A9740FF00F744024AB
:0F0F48000D1206A9741FF090E740EFF01206B1EA
:010F57002277
:100B390090E6B9E01208C30B80100B80110BA314C7
:100B49000BF7150B6E280B682E0B623C0B7A3F0BCB
:100B590074A20B74A300000C17120225020C1912BF
:100B69000CF0020C19121103020C19120915020CCE
:100B790019120EB8020C1990E6B8E030E70912070D
:100B8900ED12000E020C0F1206B690E6A0E020E16D
:100B9900F91207ED121AF3020C19E4F52B748925E1
:100BA9002B1206E0E0FF7440252B1206A9120787D5
:100BB900B404EAE4F52B7491252B12077DE0FF7448
:100BC90044252BF582E434E7120785B404E8E4F5FB
:100BD9002B748D252B120761E0FF7448252BF582B4
:100BE900E434E7120785B404E8121B238018E4F5FE
:100BF9002B7465252B12073FFF7440252B1206A97C
:100C0900120787B404EB1206B11207C98002C32286
:010C1900D307
:010C1A0022B7
:101A4E00C0E0C083C08290E6B5E04401F0D201123E
:0C1A5E00072A7401F0D082D083D0E0325F
:101B8900C0E0C083C08212072A7404F0D082D083D7
:031B9900D0E03267
:101B9C00C0E0C083C08212072A7402F0D082D083C6
:031BAC00D0E03254
:10198D00C0E0C083C08290E680E030E7051207AF6B
:10199D0080031207BC12072A7410F0D082D083D0B6
:0219AD00E03226
:101B3900C0E0C083C082D20312072A7408F0D082A1
:051B4900D083D0E03262
:1019AF00C0E0C083C08290E680E030E7051207AF49
:1019BF0080031207BC12072A7420F0D082D083D084
:0219CF00E03204
:011C8A003227
:011C8B003226
:011C8C003225
:011C8D003224
:011C8E003223
:011C8F003222
:011C90003221
:011C91003220
:011C9200321F
:011C9300321E
:011C9400321D
:011C9500321C
:011C9600321B
:011C9700321A
:011C98003219
:011C99003218
:011C9A003217
:011C9B003216
:011C9C003215
:011C9D003214
:011C9E003213
:011C9F003212
:011CA0003211
:011CA1003210
:011CA200320F
:011CA300320E
:011CA400320D
:011CA500320C
:011CA600320B
:011CA700320A
:011CA8003209
:011CA9003208
:011CAA003207
:011CAB003206
:011CAC003205
:011CAD003204
:0A1C190000010202030304040505A4
:1017EE00EC4EFEED4F2419F582741C3EF583E49306
:1017FE00FF3395E0FEEF24A1FFEE34E68F82F583F2
:10180E002290E6BCE0547EFF7E00E0D394807C0004
:01181E0022A7
:03000B0002146C70
:10146C00C0E0C0F0C0D075D000C000C004C005C042
:10147C0006C0070508E508B4060B0557E5577002CA
:10148C000556750800AE56AF577C007D0A12086EE3
:10149C00ED4C7008050CE50C7002050BD007D0065E
:0D14AC00D005D004D000D0D0D0F0D0E03278
:100F5800E4F529F528F527F526C203C200C202C226
:100F6800011214B9750D01750E0075150175161469
:100F7800750901750A2075130175144275170175F5
:100F88001864D2E843D82090E668E04409F090E677
:100F98005CE0443DF0D2AFD20712181F90E680E023
:100FA80054F7F0538EF8C2033001051204F6C2015B
:100FB800300329121C0E5024C203121922200016D5
:100FC80090E682E030E704E020E1EF90E682E0304E
:100FD800E604E020E0E412184E121C7B121A30805E
:010FE800C741
:1004F60090E6B9E070030205A71470030205FB2419
:10050600FE700302065524FB70030205A114700356
:1005160002059B1460731460762405600302068C42
:10052600121C7D400302069890E6BBE024FE602282
:1005360014603324FD601114602224067048E50D12
:1005460090E6B3F0E50E8037E51590E6B3F0E516D4
:10055600802DE50F90E6B3F0E5108023E51190E6D7
:10056600B3F0E512801990E6BAE0FF12187AAA06EF
:10057600A9077B01EA494B600DEE90E6B3F0EF90D8
:10058600E6B4F0020698020691121C47020698127B
:1005960000F8020698120003020698121C3E020694
:1005A60098121C7F400302069890E6B8E0247F600C
:1005B600151460192402703AA200E43325E0FFA264
:1005C60002E4334F8018E490E740F0801612180FCB
:1005D60040047D0180027D001217EEE0540190E791
:1005E60040F0E4A3F090E68AF090E68B7402F00205
:1005F6000698020691121C81400302069890E6B8FE
:10060600E024FE60162402600302069890E6BAE033
:10061600B40105C20002069802069190E6BAE0709F
:100626002C12180F40047D0180027D001217EEE0A7
:1006360054FEF090E6BCE05480131313541FFFE001
:10064600540F2F90E683F0E04420F08045803C1262
:100656001C83503E90E6B8E024FE601A24027032F5
:1006660090E6BAE0B40104D200802790E6BAE0B47E
:100676000202801E801512180F40047D0180027D43
:10068600001217EE80081218A6500790E6A0E04464
:0906960001F090E6A0E04480F0C0
:01069F002238
:03003300021C6B41
:041C6B0053D8EF3229
:10196A00902099EFF0F5CB8FCDAF05A3EFF0F5CA34
:10197A008FCCE4F5C8758E19D2BDD2AFD2ADD2CA1A
:03198A00F55A22E9
:0D1C0100902003E0FF902002E0FD02196A30
:031C7800AF5A223E
:101BD300AD07AC06C3E49DFBE49CFFEBFD02196A71
:05002E00C2CAC2AD22B0
:03002B000211F0CF
:1011F000C0E0C0F0C083C082C0D075D000C000C0C5
:1012000001C002C003C004C005C006C0079020068C
:10121000E06003121254902008E06003121545901C
:10122000201AE0600312118B90205CE0600990208E
:101230001BE060031213C8C2CFD007D006D005D080
:1012400004D003D002D001D000D0D0D082D083D03F
:04125000F0D0E032C8
:10184E0090E682E030E004E020E60B90E682E030A5
:10185E00E119E030E71590E680E04401F07F147E58
:0C186E00001214FF90E680E054FEF0220F
:1019220090E682E044C0F090E681F0438701000037
:04193200000000228F
:10181F0030070990E680E0440AF0800790E680E008
:10182F004408F07FDC7E051214FF90E65D74FFF034
:0F183F0090E65FF05391EF90E680E054F7F022CF
:081C5000E4F51ED2E9D2AF2237
:10171D0090E678E020E6F9C2E990E678E04480F0C2
:10172D00EF25E090E679F090E678E030E0F990E68C
:10173D0078E04440F090E678E020E6F990E678E035
:06174D0030E1D6D2E922D2
:1017BC00A90790E678E020E6F9E51E702390E6781C
:1017CC00E04480F0E925E090E679F08D19AF03A9AB
:1017DC0007751A018A1B891CE4F51D751E01D3229D
:0217EC00C32216
:10178800A90790E678E020E6F9E51E702590E6784E
:10179800E04480F0E925E0440190E679F08D19AF46
:1017A80003A907751A018A1B891CE4F51D751E0318
:0417B800D322C32253
:03004B00020A3175
:100A3100C0E0C083C082C085C084C086758600C006
:100A4100D075D000C000C001C002C003C006C007FD
:100A510090E678E030E206751E06020B1B90E67800
:100A6100E020E10CE51E64026006751E07020B1B07
:100A7100E51E24FE605F14603624FE7003020B0C39
:100A810024FC7003020B1824086003020B1BAB1A31
:100A9100AA1BA91CAF1D051D8F8275830012080DAD
:100AA10090E679F0E51D65197070751E05806B90F3
:100AB100E679E0AB1AAA1BA91CAE1D8E82758300D4
:100AC10012084C751E02E5196401704E90E678E03B
:100AD1004420F08045E51924FEB51D0790E678E035
:100AE1004420F0E51914B51D0A90E678E04440F081
:100AF100751E0090E679E0AB1AAA1BA91CAE1D8EEB
:100B01008275830012084C051D800F90E678E04441
:100B110040F0751E008003751E005391DFD007D091
:100B210006D003D002D001D000D0D0D086D084D05E
:080B310085D082D083D0E032B0
:02187A00A907BC
:10187C00AE17AF188F828E83A3E064037017AD018F
:10188C0019ED7001228F828E83E07C002FFDEC3EDF
:09189C00FEAF0580DF7E007F0035
:0118A5002220
:101A6A00121788E51E24FA600E146006240770F324
:0C1A7A00D322E4F51ED322E4F51ED32293
:101A86001217BCE51E24FA600E146006240770F3D4
:0C1A9600D322E4F51ED322E4F51ED32277
:1014FF008E2A8F2B90E600E054187012E52B2401F2
:10150F00FFE4352AC313F52AEF13F52B801590E668
:10151F0000E05418FFBF100BE52B25E0F52BE52A53
:10152F0033F52AE52B152BAE2A7002152A4E6005CE
:06153F0012193680EE22B5
:101936007400F58690FDA57C05A3E582458370F9C4
:01194600227E
:03004300020E00AA
:03005300020E009A
:100E0000021A4E00021B9C00021B8900021B3900C3
:100E100002198D000219AF00021C8A00021C8B000F
:100E2000021C8C00021C8D00021C8E00021C8F0014
:100E3000021C9000021C9100021C9200021C9300F4
:100E4000021C9400021C8B00021C9500021C9600E0
:100E5000021C9700021C9800021C9900021C9A00B8
:100E6000021C9B00021C8B00021C8B00021C8B00CE
:100E7000021C9C00021C9D00021C9E00021C9F0084
:100E8000021CA000021CA100021CA200021CA30064
:100E9000021CA400021CA500021CA600021CA70044
:100EA000021CA800021CA900021CAA00021CAB0024
:080EB000021CAC00021CAD00A5
:0300000002107774
:0C107700787FE4F6D8FD75815B0210BEA6
:1007F400BB010689828A83E0225002E722BBFE0203
:09080400E32289828A83E4932235
:10080D00BB010CE58229F582E5833AF583E02250A0
:10081D0006E92582F8E622BBFE06E92582F8E222EA
:0D082D00E58229F582E5833AF583E4932204
:10083A00BB010689828A83F0225002F722BBFE019D
:02084A00F32297
:10084C00F8BB010DE58229F582E5833AF583E8F0E2
:10085C00225006E92582C8F622BBFE05E92582C88E
:02086C00F22276
:10086E00BC000BBE0029EF8DF084FFADF022E4CC6E
:10087E00F875F008EF2FFFEE33FEEC33FCEE9DEC37
:10088E00984005FCEE9DFE0FD5F0E9E4CEFD22ED7D
:10089E00F8F5F0EE8420D21CFEADF075F008EF2FC7
:1008AE00FFED33FD4007985006D5F0F222C398FDB8
:0508BE000FD5F0EA2255
:1008C300D083D082F8E4937012740193700DA3A3C4
:1008D30093F8740193F5828883E4737402936860D8
:0608E300EFA3A3A380DFD8
:10141A008B2F8A308931E4F537F538E5361536AE43
:10142A0035700215354E6033AB32AA33A934120730
:10143A00F4FFAB2FAA30A9310538E538AC37700272
:10144A00053714F5828C83EF12084CEF60CD7401D6
:10145A002534F534E43533F53380C0AB2FAA30A9EF
:02146A0031222D
:101B4E00E4FFFE1207F4600C0FEF70010E09E9704E
:051B5E00F20A80EF22F5
:1008E900EF4E6012EF60010EEDBB010B89828A8326
:1008F900F0A3DFFCDEFA2289F05007F709DFFCA933
:0C090900F022BBFEFCF309DFFCA9F02289
:10108300020F58E493A3F8E493A34003F68001F21C
:1010930008DFF48029E493A3F85407240CC8C3336E
:1010A300C4540F4420C8834004F456800146F6DF3D
:1010B300E4800B0102040810204080901BC1E47EF1
:1010C300019360BCA3FF543F30E509541FFEE49332
:1010D300A360010ECF54C025E060A840B8E493A3F9
:1010E300FAE493A3F8E493A3C8C582C8CAC583CA24
:1010F300F0A3C8C582C8CAC583CADFE9DEE780BEDC
:011BD2000012
:00000001FF
